Microchip MPLAB XC8 Compiler V2.32

Linker command line:

-W-3 --edf=C:\Program Files\Microchip\xc8\v2.32\pic\dat\en_msgs.txt -cn \
  -h+dist/default/production\numberlock_with_motor_control.X.production.sym \
  --cmf=dist/default/production\numberlock_with_motor_control.X.production.cmf \
  -z -Q18F4580 -oC:\Users\Dell7270\AppData\Local\Temp\xcAs1f8.4 \
  --defsym=__MPLAB_BUILD=1 \
  -Mdist/default/production/numberlock_with_motor_control.X.production.map \
  -E1 -ver=XC8 Compiler --acfsm=1493 -ASTACK=07Dh-05FFh -pstack=STACK \
  -ACODE=00h-07FFFh -ACONST=00h-07FFFh -ASMALLCONST=0600h-06FFhx122 \
  -AMEDIUMCONST=0600h-07FFFh -ACOMRAM=01h-05Fh -AABS1=00h-05FFh \
  -ABIGRAM=01h-05FFh -ARAM=060h-0FFh,0100h-01FFhx5 -ABANK0=060h-0FFh \
  -ABANK1=0100h-01FFh -ABANK2=0200h-02FFh -ABANK3=0300h-03FFh \
  -ABANK4=0400h-04FFh -ABANK5=0500h-05FFh \
  -ASFR=0D00h-0DFFhx2,0F00h-0F5Fh,0F60h-0FFFh -ACONFIG=0300000h-030000Dh \
  -AIDLOC=0200000h-0200007h -AEEDATA=0F00000h-0F000FFh -peeprom_data=EEDATA \
  -preset_vec=00h,intcode,intcodelo,powerup,init -pramtop=0600h \
  -psmallconst=SMALLCONST -pmediumconst=MEDIUMCONST -pconst=CONST \
  -AFARRAM=00h-00h \
  -prdata=COMRAM,nvrram=COMRAM,nvbit=COMRAM,rbss=COMRAM,rbit=COMRAM \
  -pfarbss=FARRAM,fardata=FARRAM,nvFARRAM=FARRAM \
  -pintsave_regs=BIGRAM,bigbss=BIGRAM,bigdata=BIGRAM -pbss=RAM \
  -pidata=CODE,irdata=CODE,ibigdata=CODE,ifardata=CODE -prparam=COMRAM \
  C:\Users\Dell7270\AppData\Local\Temp\xcAs1f8.o \
  dist/default/production\numberlock_with_motor_control.X.production.o 

Object code version is 3.11

Machine type is 18F4580



                Name                               Link     Load   Length Selector   Space Scale
C:\Users\Dell7270\AppData\Local\Temp\xcAs1f8.o
                idloc                            200000   200000        8        0       5
                config                           300000   300000        E        0       4
                init                                  0        0        4        0       0
dist/default/production\numberlock_with_motor_control.X.production.o
                idloc                            200000   200000        8        0       5
                config                           300000   300000        E        0       4
                text5                              7BE2     7BE2       30     3DF1       0
                text4                              7BBC     7BBC       26     3DDE       0
                text3                              7C42     7C42       3A     3E21       0
                text2                              7C12     7C12       30     3E09       0
                text1                              7E56     7E56      1AA     3F2B       0
                text0                              7CC6     7CC6      190     3E63       0
                cstackCOMRAM                          1        1       43        1       1
                dataBANK0                            60       60       1D       60       1
                dataCOMRAM                           44       44       12        1       1
                cinit                              7C7C     7C7C       4A     3E3E       0
                idataBANK0                         7B9F     7B9F       1D     7B9F       0
                idataCOMRAM                        7B8D     7B8D       12     7B8D       0

TOTAL           Name                               Link     Load   Length     Space
        CLASS   STACK          

        CLASS   CODE           
                init                                  0        0        4         0
                text5                              7BE2     7BE2       30         0
                text4                              7BBC     7BBC       26         0
                text3                              7C42     7C42       3A         0
                text2                              7C12     7C12       30         0
                text1                              7E56     7E56      1AA         0
                text0                              7CC6     7CC6      190         0
                cinit                              7C7C     7C7C       4A         0
                idataBANK0                         7B9F     7B9F       1D         0
                idataCOMRAM                        7B8D     7B8D       12         0

        CLASS   CONST          

        CLASS   SMALLCONST     

        CLASS   MEDIUMCONST    

        CLASS   COMRAM         
                cstackCOMRAM                          1        1       43         1
                dataCOMRAM                           44       44       12         1

        CLASS   ABS1           

        CLASS   BIGRAM         

        CLASS   RAM            

        CLASS   BANK0          
                dataBANK0                            60       60       1D         1

        CLASS   BANK1          

        CLASS   BANK2          

        CLASS   BANK3          

        CLASS   BANK4          

        CLASS   BANK5          

        CLASS   SFR            

        CLASS   CONFIG         
                config                           300000   300000        E         4

        CLASS   IDLOC          
                idloc                            200000   200000        8         5

        CLASS   EEDATA         

        CLASS   FARRAM         



SEGMENTS        Name                           Load    Length   Top    Selector   Space  Class

                reset_vec                      000000  000004  000004         0       0  CODE    
                cstackCOMRAM                   000001  000055  000056         1       1  COMRAM  
                dataBANK0                      000060  00001D  00007D        60       1  BANK0   
                idataCOMRAM                    007B8D  000012  007B9F      7B8D       0  CODE    
                idataBANK0                     007B9F  00001D  007BBC      7B9F       0  CODE    
                text4                          007BBC  000026  007BE2      3DDE       0  CODE    
                text5                          007BE2  000030  007C12      3DF1       0  CODE    
                text2                          007C12  000030  007C42      3E09       0  CODE    
                text3                          007C42  00003A  007C7C      3E21       0  CODE    
                cinit                          007C7C  00004A  007CC6      3E3E       0  CODE    
                text0                          007CC6  000190  007E56      3E63       0  CODE    
                text1                          007E56  0001AA  008000      3F2B       0  CODE    


UNUSED ADDRESS RANGES

        Name                Unused          Largest block    Delta
        BANK0            00007D-0000FF               83
        BANK1            000100-0001FF              100
        BANK2            000200-0002FF              100
        BANK3            000300-0003FF              100
        BANK4            000400-0004FF              100
        BANK5            000500-0005FF              100
        BIGRAM           000056-00005F                A
                         00007D-0005FF              583
        CODE             000004-007B8C             7B89
        COMRAM           000056-00005F                A
        CONST            000004-007B8C             7B89
        EEDATA           F00000-F000FF              100
        MEDIUMCONST      000600-007B8C             758D
        RAM              00007D-0005FF              100
        SFR              000D00-000FFF              100
        SMALLCONST       000600-007B8C              100
        STACK            00007D-0005FF              583

                                  Symbol Table

_PORTB                   (abs)        000F81
_PORTD                   (abs)        000F83
_RA0                     (abs)        007C00
_RA1                     (abs)        007C01
_RA2                     (abs)        007C02
_RC0                     (abs)        007C10
_RC1                     (abs)        007C11
_TRISA                   (abs)        000F92
_TRISB                   (abs)        000F93
_TRISC                   (abs)        000F94
_TRISD                   (abs)        000F95
__HRAM                   (abs)        000000
__Habs1                  abs1         000000
__Hbank0                 bank0        000000
__Hbank1                 bank1        000000
__Hbank2                 bank2        000000
__Hbank3                 bank3        000000
__Hbank4                 bank4        000000
__Hbank5                 bank5        000000
__Hbigbss                bigbss       000000
__Hbigdata               bigdata      000000
__Hbigram                bigram       000000
__Hbss                   bss          000000
__Hcinit                 cinit        000000
__Hclrtext               clrtext      000000
__Hcomram                comram       000000
__Hconfig                config       30000E
__Hconst                 const        000000
__HcstackCOMRAM          cstackCOMRAM 000000
__Hdata                  data         000000
__HdataBANK0             dataBANK0    000000
__HdataCOMRAM            dataCOMRAM   000000
__Heeprom_data           eeprom_data  000000
__Hfarbss                farbss       000000
__Hfardata               fardata      000000
__Hibigdata              ibigdata     000000
__Hidata                 idata        000000
__HidataBANK0            idataBANK0   000000
__HidataCOMRAM           idataCOMRAM  000000
__Hidloc                 idloc        200008
__Hifardata              ifardata     000000
__Hinit                  init         000004
__Hintcode               intcode      000000
__Hintcode_body          intcode_body 000000
__Hintcodelo             intcodelo    000000
__Hintentry              intentry     000000
__Hintret                intret       000000
__Hintsave_regs          intsave_regs 000000
__Hirdata                irdata       000000
__Hmediumconst           mediumconst  000000
__HnvFARRAM              nvFARRAM     000000
__Hnvbit                 nvbit        000000
__Hnvrram                nvrram       000000
__Hparam                 rparam       000000
__Hpowerup               powerup      000000
__Hram                   ram          000000
__Hramtop                ramtop       000600
__Hrbit                  rbit         000000
__Hrbss                  rbss         000000
__Hrdata                 rdata        000000
__Hreset_vec             reset_vec    000000
__Hrparam                rparam       000000
__Hsfr                   sfr          000000
__Hsmallconst            smallconst   000000
__Hspace_0               (abs)        008000
__Hspace_1               (abs)        00007D
__Hspace_2               (abs)        000000
__Hspace_4               (abs)        60000E
__Hstack                 stack        000000
__Hstruct                struct       000000
__Htemp                  temp         000000
__Htext                  text         000000
__Htext0                 text0        000000
__Htext1                 text1        000000
__Htext2                 text2        000000
__Htext3                 text3        000000
__Htext4                 text4        000000
__Htext5                 text5        000000
__LRAM                   (abs)        000001
__Labs1                  abs1         000000
__Lbank0                 bank0        000000
__Lbank1                 bank1        000000
__Lbank2                 bank2        000000
__Lbank3                 bank3        000000
__Lbank4                 bank4        000000
__Lbank5                 bank5        000000
__Lbigbss                bigbss       000000
__Lbigdata               bigdata      000000
__Lbigram                bigram       000000
__Lbss                   bss          000000
__Lcinit                 cinit        000000
__Lclrtext               clrtext      000000
__Lcomram                comram       000000
__Lconfig                config       000000
__Lconst                 const        000000
__LcstackCOMRAM          cstackCOMRAM 000000
__Ldata                  data         000000
__LdataBANK0             dataBANK0    000000
__LdataCOMRAM            dataCOMRAM   000000
__Leeprom_data           eeprom_data  000000
__Lfarbss                farbss       000000
__Lfardata               fardata      000000
__Libigdata              ibigdata     000000
__Lidata                 idata        000000
__LidataBANK0            idataBANK0   000000
__LidataCOMRAM           idataCOMRAM  000000
__Lidloc                 idloc        000000
__Lifardata              ifardata     000000
__Linit                  init         000000
__Lintcode               intcode      000000
__Lintcode_body          intcode_body 000000
__Lintcodelo             intcodelo    000000
__Lintentry              intentry     000000
__Lintret                intret       000000
__Lintsave_regs          intsave_regs 000000
__Lirdata                irdata       000000
__Lmediumconst           mediumconst  000000
__LnvFARRAM              nvFARRAM     000000
__Lnvbit                 nvbit        000000
__Lnvrram                nvrram       000000
__Lparam                 rparam       000000
__Lpowerup               powerup      000000
__Lram                   ram          000000
__Lramtop                ramtop       000600
__Lrbit                  rbit         000000
__Lrbss                  rbss         000000
__Lrdata                 rdata        000000
__Lreset_vec             reset_vec    000000
__Lrparam                rparam       000000
__Lsfr                   sfr          000000
__Lsmallconst            smallconst   000000
__Lspace_0               (abs)        000000
__Lspace_1               (abs)        000000
__Lspace_2               (abs)        000000
__Lspace_4               (abs)        000000
__Lstack                 stack        000000
__Lstruct                struct       000000
__Ltemp                  temp         000000
__Ltext                  text         000000
__Ltext0                 text0        000000
__Ltext1                 text1        000000
__Ltext2                 text2        000000
__Ltext3                 text3        000000
__Ltext4                 text4        000000
__Ltext5                 text5        000000
__S0                     (abs)        008000
__S1                     (abs)        00007D
__S2                     (abs)        000000
__S4                     (abs)        000000
__S5                     (abs)        000000
___inthi_sp              stack        000000
___intlo_sp              stack        000000
___param_bank            (abs)        000000
___rparam_used           (abs)        000001
___sp                    stack        000000
__accesstop              (abs)        000060
__activetblptr           (abs)        000002
__end_of__initialization cinit        007CBC
__end_of_command         text4        007BE2
__end_of_data            text3        007C7C
__end_of_delay           text5        007C12
__end_of_display         text2        007C42
__end_of_keypad          text1        008000
__end_of_main            text0        007E56
__initialization         cinit        007C7C
__mediumconst            mediumconst  000000
__pcinit                 cinit        007C7C
__pcstackCOMRAM          cstackCOMRAM 000001
__pdataBANK0             dataBANK0    000060
__pdataCOMRAM            dataCOMRAM   000044
__pidataBANK0            idataBANK0   007B9F
__pidataCOMRAM           idataCOMRAM  007B8D
__ptext0                 text0        007CC6
__ptext1                 text1        007E56
__ptext2                 text2        007C12
__ptext3                 text3        007C42
__ptext4                 text4        007BBC
__ptext5                 text5        007BE2
__ramtop                 ramtop       000600
__size_of_command        (abs)        000000
__size_of_data           (abs)        000000
__size_of_delay          (abs)        000000
__size_of_display        (abs)        000000
__size_of_keypad         (abs)        000000
__size_of_main           (abs)        000000
__smallconst             smallconst   000000
_command                 text4        007BBC
_data                    text3        007C42
_delay                   text5        007BE2
_display                 text2        007C12
_keypad                  text1        007E56
_main                    text0        007CC6
command@c                cstackCOMRAM 000006
data@b                   cstackCOMRAM 000006
delay@i                  cstackCOMRAM 000004
delay@ms                 cstackCOMRAM 000001
display@p                cstackCOMRAM 000007
end_of_initialization    cinit        007CBC
intlevel0                text         000000
intlevel1                text         000000
intlevel2                text         000000
intlevel3                text         000000
isa$std                  (abs)        000001
isa$xinst                (abs)        000000
keypad@a                 cstackCOMRAM 000003
main@F10439              dataCOMRAM   000052
main@F10442              dataBANK0    000060
main@F10444              dataCOMRAM   000044
main@F10446              dataBANK0    00006F
main@arr1                cstackCOMRAM 00000B
main@arr2                cstackCOMRAM 00001A
main@arr3                cstackCOMRAM 000028
main@b                   cstackCOMRAM 00003E
main@p                   cstackCOMRAM 000040
main@p_77                cstackCOMRAM 000042
main@realpass            cstackCOMRAM 000036
main@user                cstackCOMRAM 00003A
stackhi                  (abs)        0005FF
stacklo                  (abs)        00007D
start                    init         000000
start_initialization     cinit        007C7C


MODULE INFORMATION

Module		Function		Class		Link	Load	Size
numberlock with motor control.c
		_delay         		CODE           	7BE2	0000	48
		_display       		CODE           	7C12	0000	48
		_main          		CODE           	7CC6	0000	400
		_keypad        		CODE           	7E56	0000	426
		_data          		CODE           	7C42	0000	58
		_command       		CODE           	7BBC	0000	38

numberlock with motor control.c estimated size: 1018

shared
		__initialization		CODE           	7C7C	0000	64

shared estimated size: 64

